:100000004528A00014200C080D04031940283A20AC
:1000100084132008800664000D280E288C0A03191A
:100020008D0F0B2880064028FF3A84178005402852
:100030008F018E00FF308E07031C8F07031C4028A2
:1000400003308D00DF3026201A288D01E83E8C0019
:100050008D09FC30031C2F288C0703182C288C07D3
:1000600064008D0F2C280C1835288C1C39280000B2
:10007000392808008C098D098C0A03198D0A08009B
:100080008313031383126400080086130613861279
:100090008C30A5008C30A4008C30A6000130A70065
:1000A00064000830270203186728AA30A500B3208F
:1000B000A030A400A030A600B3206430A500B32077
:1000C0007830A4007830A600B320A70F5028013064
:1000D000A70064000430270203188028AA30A50076
:1000E000B3207830A400A030A600B3206430A5006F
:1000F000B320A030A4007830A600B320A70F692851
:100100000130A70064000830270203189928AA309C
:10011000A500B3207830A4007830A600B320643066
:10012000A500B320A030A400A030A600B320A70FE4
:1001300082280130A7006400043027020318B22887
:10014000AA30A500B320A030A4007830A600B320C8
:100150006430A500B3207830A400A030A600B320FE
:10016000A70F9B284E280130A80064000B302802FE
:100170000318D32825088C008D01063084008030B8
:10018000012024088C008D010630840040300120BD
:1001900026088C008D0106308400203001200D30AF
:0C01A0001820A80FB52808006300D42820
:02400E00F53F7C
:00000001FF
